:101E18002020202020200D0A002A56455253494FE1
:101E28004E3A20522D4441532056322E340D0A008A
:101E38002A4D4553534147453A2053656C667465AE
:101E48007374207061737365640D0A002A574152D8
:101E58004E494E473A2053656C6674657374206624
:101E680061696C65640D0A002A52454144590D0A9E
:101E780000000000002A01005202007903009E04BD
:101E880000C20500E5060106070127080146090109
:101E9800640A01E90F02581403001E03742803C3DF
:071EA8003203F93C04023E85
:100CA3009070F0EEF0A3EFF0A37401F09070F2E017
:100CB300FF6412602AEF75F003A42479F582E4340B
:100CC3001EF583E493FC740193FDC39070F1E09DE2
:100CD3009070F0E09C40089070F2E004F080CDEF5B
:100CE30075F003A42479F582E4341EF583E493FEBE
:100CF300740193FF9070F0E0FCA3E0FDC3EF9DFF50
:100D0300EE9CFEE4FCFDC8ECC8C9EDC9CAEECACB33
:100D1300EFCBA3E075F003A42478F582E4341EF549
:100D230083E493FFE4FE1204C0ECC0E0EDC0E0EE08
:100D3300C0E0EFC0E09070F2E075F003A42476F514
:100D430082E4341EF583E493FE740193FFC3907031
:100D5300F1E09FFF9070F0E09EFEE4FCFDC8ECC85C
:100D6300C9EDC9CAEECACBEFCB9070F2E075F003C0
:100D7300A4247BF582E4341EF583E493FFE4FE129E
:100D830004C0D0E0FBD0E0FAD0E0F9D0E0F8EF2BDC
:100D9300FFEE3AFEED39FDEC38FC9070F3120617C6
:100DA3007FE87E037D007C009070F3E0F8A3E0F918
:100DB300A3E0FAA3E0FB1204C0C8ECC8C9EDC9CA9A
:100DC300EECACBEFCB9070F2E0FF75F003A424766C
:100DD300F582E4341EF583E493FC740193FDEF750F
:100DE300F003A42479F582E4341EF583C3740193DC
:100DF3009DFFE4939CC313FEEF13FFE4FCFDEB2F75
:100E0300FFEA3EFEED39FDEC38FCECC0E0EDC0E05E
:100E1300EEC0E0EFC0E09070F2E0FF75F003A424B1
:100E230076F582E4341EF583E493FC740193FDEFBD
:100E330075F003A42479F582E4341EF583C37401A9
:100E4300939DFFE4939CFEE4FCFDF8F9CAEECACB44
:100E5300EFCBD0E0FFD0E0FED0E0FDD0E0FC120508
:020E63004B2220
:1016A700301503021744E56164036009E561640BC3
:1016B70060030217A9C3E54F78CF96FFE54E18964A
:1016C700FE120CA3CBEFCBCAEECAEB4A7003FA7B30
:1016D70001D201E49070E9F0CEEACECFEBCF7C00E7
:1016E7007D0A1204099070E9E024EAF582E4347077
:1016F700F583EDF0CEEACECFEBCF7C007D0A120466
:1017070009CAEECACBEFCB9070E9E004F0E0B4056C
:10171700C79070E97404F09070E9E0FFF460157405
:10172700EA2FF582E43470F583E070089070E9E001
:1017370014F080E3EF049070EFF0D215227F1E12B1
:101747002C687F017D327B04122D40301304301743
:10175700FA227F0A122C689070EFE0149070E9F07B
:101767009070E9E024EAF582E43470F583E0700BC9
:101777007F017D0B7B04122D4080169070E9E024D9
:10178700EAF582E43470F583E0FF7D0B7B01122DCF
:10179700403013043017FA229070E9E0FF14F0EF9D
:0317A70070BE22EF
:10206E00D2AF122B76122C8B122C03122BA8122D00
:10207E0074122CF0122D341222467BFF7A1E791820
:10208E001200C97BFF7A1E79211200C912285D50F9
:10209E00107BFF7A1E79381200C97F01122D16802F
:1020AE00097BFF7A1E79541200C9121F469070A444
:1020BE00E0FF1227EB122A1312257F9070A5E0FE87
:1020CE00A3E0FF1226EE7BFF7A1E79701200C9C2C2
:0D20DE0015301703122B901216A780F52263
:03000B000221D7F8
:1021D700C0E0C0F0C083C082C0D075D008C28CAF49
:1021E7008CEFFEAD8AED255878D1F6E5573E18F607
:1021F700F58C08E6F58AD28CD55C0990709BE0F5E2
:102207005C1224BDD55B1B90709BE0F55B055AE51E
:102217005A70020559E55A45597007E5616003751B
:102227006105E5616404600C1218AC12245A121C93
:0F2237000E121FDAD0D0D082D083D0F0D0E03298
:1026EE00E4FCFDFB7AC079A8F81204C07BE07A2ED8
:1026FE00790078001226AAC374129FF558E49EF54D
:10270E005790709BE0F55CF55BE4F559F55AE58959
:10271E0054F04401F589758CFF758AFFC2B9D2A9B0
:03272E00D28C2228
:0C2CB60090709BE0F55BE4F559F55A22A4
:10257F00E5C520E3FB75C50775C50FE5C530E4FB61
:10258F00AFC6EF75F004A4FFAEF0E5C5C413135446
:10259F00037C002FF53CEC3EF53BE4F53AE53A259C
:1025AF00E024BAF8A63B08A63CE53C2527F527E52D
:1025BF003B3526F526053AE53AB40AE1E4F539222A
:1018AC00C0D075D0083016030219A8E5C520E3FB9B
:1018BC00E4F5C575C508F543754401E54364087046
:1018CC0003021987E5C530E4FB85C62885C53DE5CF
:1018DC00436407600EE5C520E3FBE54304F5C5440E
:1018EC0008F5C5E52875F004A4FFAEF0E53DC4137A
:1018FC001354037C002FF546EC3EF545E54325E0FB
:10190C002429F8A64508A64690709AE055446060D4
:10191C00AF28122900AF3D122900E543B406088513
:10192C0045418546428049E54364077043E53925C6
:10193C00E024BBF8C3E52796F527E5261896F5268F
:10194C00E53925E024BAF8A64508A646E54625273C
:10195C00F527E5453526F526FEAF277C007D0A12D6
:10196C0004098E248F250539E539B40A03E4F539C9
:10197C000543E54425E0F5440218C7300F1EE4A2E8
:10198C00C492E4A2C592E5A29692E6A29792E725AC
:0F199C0061C4F53EAF3E122900853E40D0D022F7
:10216700C0D075D008300F659070A4E0FD7C00905A
:1021770070ACE0FB24FFFFE434FFFE1203F5EF240D
:1021870001FFE43EFEC3E51F9FF51FE51E9EF51EFA
:102197008B3FE53F6021E51EF583E51FF582E0C42F
:1021A70054F02561C4F09070A4E0251FF51FE435B5
:1021B7001EF51E153F80DB9070A4E024FFFFE4347A
:1021C700FFFEC3E51F9FF51FE51E9EF51ED0D0221B
:0D2CA900E4F56FF570F571C21612282422B3
:10245A00C0D075D008E5616057201654122C55403B
:10246A004F9070A4E025E09070E6F09070E6E0608E
:10247A003F20113C1229348F6E12002E0570E57030
:10248A007002056F7004E56F6480701CF56FF5705B
:10249A000571E571B40C04D2168015122C42E5714F
:1024AA0020E00512282480089070E6E014F080BB32
:0324BA00D0D0225D
:102A1300E4907133F0A3F090712F120623000000AD
:102A23000074FF78CEF608F6E4907135F0F562F5A0
:082A33006190712E74FFF02286
:10000E00C0D075D008756101C290122CA97F021262
:05001E002D16D0D022D8
:102BD700C0D0C291E55A240190712DF0E435599087
:062BE700712CF0D0D02299
:102BED00C0D0C292E55A240190712DF0E435599070
:062BFD00712CF0D0D02283
:10145500C0D075D008E49070E6F020C604E04401E1
:10146500F020C7079070E6E04402F090712EE0FF8F
:101475009070E6E0FE6F603BEE702590713BE0FFFB
:101485006005122D1E802C90713AE0FF6403600404
:10149500EFB40405122D1E801A7F01122D1680133C
:1014A5009070E6E030E0077F01122D1E80057F0277
:1014B500122D1E9070E6E090712EF0300B1EA29456
:1014C500300C01B34016C218122CB6907098E0FE8D
:1014D500A3E0FF12296812000E02159620100302E0
:1014E5001596907097E0C4F8540FC868FF907096F1
:1014F500E0C454F048FEC3E54D9FFDE54C9EFCE578
:1015050042C4F8540FC868FFE541C454F048FED3FF
:10151500EF9DEE9C4016D21890712F120623000005
:101525000000E4907133F0122CB68065C2189071FA
:101535002FE0F8A3E0F9A3E0FAA3E0FBE8C0E0E5BB
:1015450042C4F8540FC868FFE541C454F048FEC3CF
:10155500EF954DFFEE954CFE3395E0FDFCD0E0F8A0
:10156500EB2FFFEA3EFEE93DFDE83CFC90712F12B2
:1015750006179070ACE0FF907133E004F06F7011C6
:1015850090709FE0FEA3E0FF12296812000E122161
:0415950067D0D02229
:101EAF00C0D075D00890712FE0F8A3E0F9A3E0FA45
:101EBF00A3E0FBE8C0E0E542C4F8540FC868FFE5B3
:101ECF0041C454F048FEC3EF954DFFEE954CFE33E1
:101EDF0095E0FDFCD0E0F8EB2FFFEA3EFEE93DFD7B
:101EEF00E83CFC90712F120617300E337F007E00F6
:101EFF007D007C0090712FE0F8A3E0F9A3E0FAA336
:101F0F00E0FBD31205DD4017907095E0FFD3E55A43
:101F1F009FE55994004008122BD775610280153048
:101F2F000D129070AAE0655A7002E5597006122BD7
:071F3F00D775610AD0D02222
:10232100C0D075D00890712CE0FEA3E0655A70030F
:10233100E5596E7002D291300E379070A2E0FEA383
:10234100E0FFC3E54F9FFFE54E9EFEC3E5259FE5F8
:10235100249E5007E4907134F080169070BDE0FF28
:10236100907134E004F06F7008122BED75610380F9
:1023710015300D129070ABE0655A7002E559700688
:09238100122BED75610BD0D02286
:102B2300C0D075D00890712CE0FEA3E0655A700305
:0C2B3300E5596E7004D291D292D0D022ED
:101C0E00C0D075D008E5617003021C9CE4F55D75CB
:101C1E006001E55D64086065E55D25E024ADF58253
:101C2E00E43470F583E0FEA3E08E5EF55FF470039E
:101C3E00E55EF4603EE56255607015E55A655F70CD
:101C4E0004E559655E7009E5604262AF5D12261BC0
:101C5E00E5625560601DE55F2401FFE4355EFEEF31
:101C6E00655A7003EE6559700AE560F45262AF5D15
:101C7E00122663055DE56025E0F5608095C3E525D8
:101C8E0078CF96E52418965005A62408A625E5617A
:101C9E0014601614601814601A24F960111460137D
:101CAE00240B7012121455800D121EAF80081223D1
:091CBE00218003122B23D0D02257
:1027EB00CBEFCBEBFD7C007E407F00120409CDEBE1
:1027FB00CD7C001203F58E1A8F1B74002FF582EE21
:10280B003430AF82F5188F197E307F008E1C8F1DF0
:09281B008E1E8F1FD211C2122281
:10290000C211051FE51FAC1E7002051E14F5828C56
:1029100083EFF0E51F65197004E51E6518700675F4
:102920001E30751F00E51F651D7004E51E651C70D7
:0429300002D212229B
:10293400C212051DE51DAE1C7002051C14F5828E25
:1029440083E0FFE51D65197004E51C6518700675C4
:102954001C30751D00E51F651D7004E51E651C70A7
:0429640002D2112268
:10296800C3E51F9FF51DE51E9EF51CC3E51D9400DC
:10297800E51C9430400BD3E51D9519E51C951840CE
:0E2988000CE51B251DF51DE51A351CF51C225E
:101CC70025732025627520256275202575202575C9
:101CD70020256275202562752025632025627520E1
:101CE70025632025632025630D0A00632069676E3D
:101CF700202575202575202575202575202575201B
:101D070025752025752025750D0A006320786D69D6
:101D17007420257520256275202562750D0A002A15
:101D270056455253494F4E3A20522D44415320565F
:101D3700322E340D0A006321006320726461730040
:101D4700632069676E006320786D697400633F00E4
:101D570063006320007265736574002A4552524F11
:101D6700523A20556E6B6E6F776E20636F6D6D61A3
:051D77006E640D0A007E
:062D3400E4F579C217224C
:100AD6009070E9EBF0A3EAF0A3E9F0300B13300CC9
:100AE600089071067401F0800D9071067402F08012
:100AF60005E4907106F09070E9E0FBA3E0FAA3E04C
:100B0600F91203BA643F6003020BAE9070ECE0F991
:100B1600A3E0FAA3E09070C1C9F0A3EAF0A3E9F05C
:100B260090709BE09070C4F090709AE09070C5F061
:100B3600907096E0FFA3E09070C6CFF0A3EFF09020
:100B460070A2E0FFA3E09070C8CFF0A3EFF0907022
:100B5600AAE09070CAF09070ABE09070CBF0300FC6
:100B6600047F3180027F309070CCEFF0907106E008
:100B76009070CDF03010047F3180027F309070CEBF
:100B8600EFF0300E047F3180027F309070CFEFF0AF
:100B9600300D047F3180027F309070D0EFF07BFF04
:100BA6007A1C79C71200C9229070E9E0FBA3E0FA2B
:100BB600A3E0F91203BAFF122C2D500C9070EAE450
:100BC60075F00112049480E0E4907105F09070E9EC
:100BD600E0FBA3E0FAA3E0F91219AB907105E0255A
:100BE600E024EFF582E43470F583EEF0A3EFF090A5
:100BF60070E9E0FBA3E475F0011204AAA9F0FA1269
:100C060003BAFF122C2D50E7907105E004F0E0B412
:100C16000BBB9070F0E090709BF09070F2E09070DB
:100C26009AF09070F3E0FFA3E0907096CFF0A3EFF8
:100C3600F09070F5E0FFA3E09070A2CFF0A3EFF084
:100C46009070F8E09070AAF09070FAE09070ABF0B7
:100C56009070FBE0FEA3E0FFEE4F24FF920FA3E0AF
:100C6600FEA3E0FFEE4F24FF920BEF64014E7003EC
:100C7600D38001C3920C9070FFE0FEA3E0FFEE4F1D
:100C860024FF9210A3E0FEA3E0FFEE4F24FF920E96
:0D0C9600A3E0FEA3E0FFEE4F24FF920D222D
:1017AA009070E9EBF0A3EAF0A3E9F01203BA643F00
:1017BA0060030218417BFF7A1C79F29070ADE0FF5A
:1017CA00A3E09070C1CFF0A3EFF09070AFE0FFA359
:1017DA00E09070C3CFF0A3EFF09070B1E0FFA3E008
:1017EA009070C5CFF0A3EFF09070B3E0FFA3E09044
:1017FA0070C7CFF0A3EFF09070B5E0FFA3E0907050
:10180A00C9CFF0A3EFF09070B7E0FFA3E09070CBE0
:10181A00CFF0A3EFF09070B9E0FFA3E09070CDCFC6
:10182A00F0A3EFF09070BBE0FFA3E09070CFCFF091
:10183A00A3EFF01200C9229070E9E0FBA3E0FAA33B
:10184A00E0F91203BAFF122C2D500C9070EAE475DD
:10185A00F00112049480E0E49070ECF09070E9E0FA
:10186A00FBA3E0FAA3E0F91219AB9070ECE025E0D3
:10187A0024ADF582E43470F583EEF0A3EFF09070B6
:10188A00E9E0FBA3E475F0011204AAA9F0FA120335
:10189A00BAFF122C2D50E79070ECE004F0E0B40887
:0218AA00BB225F
:101B4A009070E9EBF0A3EAF0A3E9F01203BAB43F0C
:101B5A00297BFF7A1D791290709CE0FFA3E09070B8
:101B6A00C1CFF0A3EFF09070A9E09070C3F090702D
:101B7A009EE09070C4F01200C9229070E9E0FBA3C5
:101B8A00E0FAA3E0F91203BAFF122C2D500C907060
:101B9A00EAE475F00112049480E0E49070F2F090A7
:101BAA0070E9E0FBA3E0FAA3E0F91219AB9070F236
:101BBA00E025E024ECF582E43470F583EEF0A3EF3F
:101BCA00F09070E9E0FBA3E475F0011204AAA9F011
:101BDA00FA1203BAFF122C2D50E79070F2E004F0CB
:101BEA00E0B403BB9070ECE0FFA3E090709CCFF0F0
:101BFA00A3EFF09070EFE09070A9F09070F1E09090
:041C0A00709EF022B6
:1006F9007B017A7079577D20122B3F9070ECEBF0DB
:10070900A3EAF0A3E9F04A70047F0180027F009018
:1007190070F9EFF0605F7B017A707956121599C80C
:10072900ECC8C9EDC9CAEECACBEFCB9070A7E0FE01
:10073900A3E0FFE4FCFD1204C0C8ECC8C9EDC9CAB6
:10074900EECACBEFCB907098E0FEA3E0FFE4FCFD8E
:10075900EB2FFFEA3EFEED39FDEC38FC9070EF120D
:1007690006179070A7E0FEA3E0FFE4FCFD9070F38C
:1007790012061780767B017A707956121599C8ECA2
:10078900C8C9EDC9CAEECACBEFCB9070A4E0FFE4AB
:10079900FCFDFE1204C0C8ECC8C9EDC9CAEECACB3B
:1007A900EFCB907098E0FEA3E0FFE4FCFDEB2FFF98
:1007B900EA3EFEED39FDEC38FC9070EF1206179019
:1007C90070ECE0FBA3E0FAA3E0F9121599C8ECC8B4
:1007D900C9EDC9CAEECACBEFCB9070A4E0FFE4FC27
:1007E900FDFE1204C09070F31206179070EFE0FC42
:1007F900A3E0FDA3E0FEA3E0FF780F1206048F71CA
:100809009070EFE0FCA3E0FDA3E0FEA3E0FFEE544F
:100819007FFEE48E6F8F70122C429070F9E06009B0
:10082900E49070F7F0A3F0800B1200269070F7EEB9
:10083900F0A3EFF0E49070E9F0A3F09070E9E0FE26
:10084900A3E0FFE4FCFD9070F3E0F8A3E0F9A3E076
:10085900FAA3E0FBC31205F3606C122CC29070EB93
:10086900EFF09070F9E060149070EBE0FF9070F891
:10087900E02FF09070F7E03400F080189070F7E006
:10088900FEA3E0FF9070EBE0FD1220EB9070F7EE15
:10089900F0A3EFF09070EBE0FF1200030570E57034
:1008A9007002056F7004E56F64807009F56FF5706B
:1008B9000571122C429070EAE004F070069070E91C
:1008C900E004F00208449070F9E070139070F7E0CA
:1008D900FEA3E0FF122D2D9070F7EEF0A3EFF0903C
:1008E90070F7E0FF1200039070F8E0FF1200032296
:042D6400122A81228C
:0A2CE6007BFF7A1D79261200C92237
:10117F009070EC74FFF0A3741DF0A3743DF0A3E422
:10118F00F0A37402F07B017A7079551223F3EF709C
:10119F0004120FF8229070EC74FFF0A3741DF0A3EB
:1011AF007440F0A3E4F0A37406F07B017A707955D4
:1011BF001223F3EF70189070EC74FFF0A3741DF00E
:1011CF00A37440F07B017A70795B120AD62290707B
:1011DF00EC74FFF0A3741DF0A37447F0A3E4F0A325
:1011EF007405F07B017A7079551223F3EF700A7B47
:1011FF00017A70795A1217AA229070EC74FFF0A33B
:10120F00741DF0A3744DF0A3E4F0A37406F07B01FA
:10121F007A7079551223F3EF700A7B017A70795B3C
:10122F00121B4A229070EC74FFF0A3741DF0A3748C
:10123F0054F0A3E4F0A37402F07B017A7079551295
:10124F0023F3EF70189070EC74FFF0A3741DF0A3EC
:10125F007457F07B017A707956120AD6229070EC8F
:10126F0074FFF0A3741DF0A37459F0A3E4F0A374FA
:10127F0002F07B017A7079551223F3EF701890709A
:10128F00EC74FFF0A3741DF0A37457F07B017A7018
:10129F007956120AD622907055E0B464041206F9FA
:1012AF00229070EC74FFF0A3741DF0A3745CF0A394
:1012BF00E4F0A37405F07B017A7079551223F3EFF4
:1012CF007004122D6422907055E0B47604122CE64F
:1012DF0022907055E060097BFF7A1D79621200C978
:0112EF0022DC
:102B900010170280FB7561047F01122D167F1E1233
:082BA0002C6812117F80E9226C
:10289600C0D0EF20E72CEF640A6027EF640D6011CB
:1028A60074552579F582E43470F583EFF005798067
:1028B6001174552579F582E43470F583E4F0D21766
:0528C600F579D0D022DD
:10238A002A4D4553534147453A2053746F72696E3B
:10239A006720706172616D657465727320696E2061
:1023AA00464C4153480D0A002A4D4553534147456F
:1023BA003A2046696E69736865642073746F72693E
:1023CA006E670D0A00000001C001C802000C001B64
:1023DA000100193C03FFFFFFFFFFFFFFFFFFFFFFA5
:0923EA00FFFFFFFFFF00000003EC
:0A2CF0007575237576CF1212F022DD
:1012F0009023CFE49324FF920BA3E49324FF920C5A
:10130000A3E49324FF9210A3E49390709AF09023A7
:10131000D3E49324FF920FE49070A4F07F80EF60F9
:101320001490709AE05F60079070A4E02402F0EFE0
:10133000C313FF80E9300F069070A4E004F09023FF
:10134000D4E49390709BF09023D5E4939070A1F037
:101350009023D6E493FF740193907096CFF0A3EF9F
:10136000F09023D8E493FF7401939070A2CFF0A380
:10137000EFF090709BE0FBFD7C007E037FE81204A1
:10138000099070A5EEF0A3EFF09070A4E0FA8BF056
:10139000A4FF9070A7E5F0F0A3EFF0EB1313543F18
:1013A0009070ACF0FB9070BDF09023DAE49324FFD2
:1013B000920EA3E49324FF920DA3E4939070AAF0FD
:1013C0009023DDE4939070ABF09023DEE493907073
:1013D00095F09070A1E0FF7E009070A7E0FCA3E084
:1013E000FD1203F5907098EEF0A3EFF0EBFF7E0096
:1013F000EAFD7C001203F5E02F9070A0F090709849
:10140000E03E90709FF0E4FFEF25E024DFF582E4FA
:101410003423F583E493FC740193FDEF25E024ADC0
:10142000F582E43470F583ECF0A3EDF00FEFB4082F
:10143000D79023EFE493FF74019390709CCFF0A3B7
:10144000EFF09023F1E4939070A9F09023F2E493ED
:0514500090709EF022E7
:100FF800A20BE433857682857583F0A20CE433A3D3
:10100800F0A210E433857682857583A3A3F09070EF
:101018009AE0857682857583A3A3A3F0A20FE433B3
:10102800FFE5762404F582E43575F583EFF09070DA
:101038009BE0FFE5762405F582E43575F583EFF04E
:101048009070A1E0FFE5762406F582E43575F58316
:10105800EFF0907096E0FEA3E0FFE5762407F582B6
:10106800E43575F583EEF0A3EFF09070A2E0FEA3EF
:10107800E0FFE5762409F582E43575F583EEF0A303
:10108800EFF0A20EE433FFE576240BF582E4357524
:10109800F583EFF0A20DE433FFE576240CF582E446
:1010A8003575F583EFF09070AAE0FFE576240DF52D
:1010B80082E43575F583EFF09070ABE0FFE57624B8
:1010C8000EF582E43575F583EFF0907095E0FFE555
:1010D80076240FF582E43575F583EFF0E49070E936
:1010E800F09070E9E0FF6408603BEF25E024ADF57F
:1010F80082E43470F583E0FEA3E0FFE5762410F582
:1011080082E43575F583C083C0829070E9E0D082AF
:10111800D08375F002120654EEF0A3EFF09070E958
:10112800E004F080BC90709CE0FEA3E0FFE576242C
:1011380020F582E43575F583EEF0A3EFF09070A901
:10114800E0FFE5762422F582E43575F583EFF0902B
:10115800709EE0FFE5762423F582E43575F583EF8C
:10116800F07BFF7A23798A1200C91228CB7BFF7A99
:071178002379B21200C92225
:101F4600E5C520E3FB75C50675C50EE5C530E4FBA2
:101F5600AFC6EF75F004A4FFAEF0E5C5C413135485
:101F6600037C002FF54DEC3EF54CE5C520E3FB75F3
:101F7600C50775C50FE5C530E4FBAFC6EF75F004C0
:101F8600A4FFAEF0E5C5C4131354037C002FF54A35
:101F9600EC3EF549F54E854A4FD218E4F547F5482B
:101FA600FFEF25E0240CF582E43471F583E54CF06F
:101FB600A3E54DF0E54D2548F548E54C3547F54791
:101FC6000FEFB410DCE4F54BE5482410F54DE4358D
:041FD60047F54C225D
:1024BD0030185EE5482410F54DE43547F54CE54BF5
:1024CD0025E0240CF582E43471F583E0FEA3E0FFF2
:1024DD00C3E5489FF548E5479EF547E54B25E024C4
:1024ED000CF582E43471F583E541F0A3E542F0E5A6
:1024FD00422548F548E5413547F547054BE54BB4D1
:10250D001003E4F54B85494E854A4F8524498525B1
:02251D004A2250
:102B7600C21943878075985AE589540F4420F58910
:0A2B8600758DFFD28ED2BCD2AC22B6
:030023000229C1EE
:1029C100C0E0C0F0C083C082C0D075D0103098077D
:1029D100AF99C298122896309904C299D219D0D0D1
:0929E100D082D083D0F0D0E032A6
:080003008F993019FDC219228A
:082D0E008F993019FDC2192252
:1029EA00E5C520E3FB8FC5EF4408F5C5E5C530E42E
:1029FA00FBAFC6EF75F004A4FFAEF0E5C5C4131330
:092A0A005403FDE5F0EF4DFF223D
:102A8100E4F5A8F5E8F5B8F5F875710FE571A2E080
:102A910092B5A2E192B3A2E292B4A2E392B202FF92
:022AA100FE2213
:102C4200E571A2E092B5A2E192B3A2E292B4A2E34C
:032C520092B22219
:0C2CC200E56F4480857082F583E0FF22FE
:10002E0090D3557499F090ACAA7466F090D3557431
:10003E0090F0E56EF5F0E56FD2E7F583E570F582A9
:0D004E00E5F0F0E0A2E730F701B340F72243
:10282400E571A2E092B5A2E192B3A2E292B4A2E36E
:1028340092B290D3557499F090ACAA7466F090D388
:10284400557480F090D3557499F090ACAA7466F0E6
:092854009080007414F0D21A22E5
:102C5500301A0D908000E020E703D38001C3921A5B
:032C6500A21A228E
:1028CB0075710C122824122C5540FB75710D122CAE
:1028DB0042E4F56FF570857082856F83E0F56E12BB
:1028EB00002E0570E5707002056FE5707004E56FE2
:0528FB00648070E22280
:032D7400C21A225E
:03005B000222B5C9
:1022B500C0E0C0D0C2CC742D25C9F5C9301358155E
:1022C50050E5507052E55670128552FCC2C0F5516A
:1022D500755601E55425E0F550803CE556640170DE
:1022E5002375FCFFD2C00551E5516553700E3014BE
:1022F50007F556855550801FC213801B755602750C
:1023050050028013E556B4020E8552FCC2C07556C4
:0C23150001E55425E0F550D0D0D0E032B6
:102BA80075FCFFD2C075FE0B75528075EA0DC2FC2C
:082BB800D2EC75550AC213228C
:102A3B00C213A202921475FCFFD2C08F53E4F55659
:102A4B00CEEDCE8EFECEEBCE8E54855550EF600282
:032A5B00D2132271
:062D3A00D202122A3B2226
:062D4000C202122A3B2230
:082D16007D0B7B01122D3A2216
:082D1E007D327B04122D3A22E4
:102C6800C21375FCFFD2C08F55E4F556855550D276
:022C7800132225
:1008F9002A4D4553534147453A20615F7374203D62
:100909002025750D0A002A4D4553534147453A2084
:1009190061283029203D2025750D0A002A574152AA
:100929004E494E473A20416363656C65726174694B
:100939006F6E206F7574206F662072616E67653AFD
:1009490020615F73743D25752C2061303D2575202C
:1009590028672D7377697463682064697361626CB1
:100969006564290D0A002A4D4553534147453A20EC
:1009790070283029203D2025750D0A002A5741523B
:100989004E494E473A20507265737375726520253A
:1009990075206F7574206F662072616E6765205BC4
:1009A90025752C25755D0D0A002A5741524E494E71
:1009B900473A20427265616B776972652065727288
:1009C9006F722028425720747269676765722064C4
:1009D900697361626C6564290D0A002A5741524E98
:1009E900494E473A2049676E6974657220256264E9
:1009F90020636F6E666967757265643A20626F611C
:100A09007264206E6F7420666F756E640D0A002A19
:100A19005741524E494E473A2049676E697465728B
:100A29002025626420636F6E666967757265643A32
:100A3900206E6F20636F6E6E656374697669747971
:100A49000D0A002A5741524E494E473A20547261C5
:100A59006E736D697474657220636F6E666967750C
:100A69007265643A20626F617264206E6F742066E9
:100A79006F756E640D0A002A5741524E494E473A26
:100A89002044726F6775652069676E697465723A8B
:100A9900206E6F20636F6E6E656374697669747911
:100AA9000D0A002A5741524E494E473A204D616975
:100AB9006E2069676E697465723A206E6F20636F84
:0D0AC9006E6E65637469766974790D0A00BC
:072D2600EF60031F80FA2299
:102B0400A2029293E4F577F5787F78122D26057862
:0F2B1400E57870020577E578640A457770EB2263
:100E6500E49070EEF09070E9F0A3F09070EDF0D2A0
:100E750002122B047F061229EA9070EAE02FF09007
:100E850070E9E03EF0C202122B049070EDE004F030
:100E9500E0B420DB9070E9E0FEA3E0FF7C007D205C
:100EA50012045E9070E9EEF0A3EFF07BFF7A08790B
:100EB500F99070C1EEF0A3EFF01200C9E49070EB69
:100EC500F0A3F0A3F07F061229EA9070ECE02FF072
:100ED5009070EBE03EF09070EDE004F0E0B420E5BA
:100EE5009070EBE0FEA3E0FF7C007D2012045E9095
:100EF50070EBEEF0A3EFF07BFF7A09790F9070C1EC
:100F0500EEF0A3EFF01200C99070EBE0FEA3E0FF56
:100F15009070E9E0FCA3E0FDC39FFFEC9EFEC3EFEC
:100F2500942DEE64809480502D7BFF7A097925906D
:100F350070C1ECF0A3EDF09070EBE0FFA3E09070D2
:100F4500C3CFF0A3EFF01200C97F06122D1EC21009
:100F55009070EE7406F0E49070E9F0A3F09070EDF7
:100F6500F07F071229EA9070EAE02FF09070E9E02F
:100F75003EF09070EDE004F0E0B420E59070E9E01B
:100F8500FEA3E0FF7C007D2012045E9070E9EEF088
:100F9500A3EFF07BFF7A09796F9070C1EEF0A3EFB4
:100FA500F01200C99070E9E0FEA3E0FFC3947DEE66
:100FB50064809482400BD3EF94DBEE64809483408D
:100FC5002C7BFF7A0979859070C1EEF0A3EFF0A331
:100FD5007402F0A3747DF0A37403F0A374DBF01224
:100FE50000C97F05122D1E9070EE7405F09070EE0D
:030FF500E0FF22F8
:101A8300E49070E9F0300B1EA294300C01B34016C1
:101A93007BFF7A0979B21200C97F03122D1EC20B94
:101AA3009070E97403F0E49070EAF09070EAE0FF5C
:101AB3006408606AEF25E024ADF582E43470F583B1
:101AC300E0FCA3E0F47002ECF4604B122CCE401F58
:101AD3007F04122D1E7BFF7A0979E49070EAE004FB
:101AE3009070C1F01200C99070E97404F0802790DF
:101AF30070EAE0FF1225CF401D7F04122D1E7BFFED
:101B03007A0A79189070EAE0049070C1F01200C963
:101B13009070E97404F09070EAE004F0808D9070A6
:101B23009CE07002A3E06019122D4640147F04125A
:101B33002D1E7BFF7A0A794C1200C99070E9740458
:071B4300F09070E9E0FF22C1
:10285D00D201121A8390713AEFF06002C201120E8A
:10286D006590713BEFF06002C20120C60B7BFF7AD1
:10287D000A79801200C9C20120C70B7BFF7A0A7941
:09288D00AC1200C9C201A2012233
:102C0300E4FF74362FF582E43471F58374FFF00F1B
:052C1300EFB404EE2205
:0C2CCE00EFC31325E02441FF122B5B2212
:1025CF009070EBEFF0E0FFC31325E02441FF7B0198
:1025DF007A7079ED9070F27401F01227319070ECEF
:1025EF00EFF09070EBE054012402FF74017E00C8FD
:1025FF00EFC8088005C333CE33CED8F9FF9070ED06
:0C260F00E0FDE4EF5D6003D38001C32216
:10261B00CEEFCEEEC313FF2436F582E43471F5838F
:10262B00C083C082E0FDEE5401FC7401C8ECC80805
:10263B008002C333D8FCF45DD082D083F0EF25E069
:10264B002440FFEEC3132436F582E43471AD82FCD3
:08265B007B01D2011227B0221D
:10266300CEEFCEEEC313FF2436F582E43471F58347
:10267300C083C082E0FDEE5401FC7401C8ECC808BD
:102683008002C333D8FC4DD082D083F0EF25E02401
:1026930040FFEEC3132436F582E43471AD82FC7B34
:0726A30001D2011227B02251
:10224600E4F572F573F57490709CE0FEA3E0FF4E22
:10225600605C9070407404F0E4A3F0FCFD7BC0FA6F
:10226600F9F81204C0C8ECC8C9EDC9CAEECACBEF6A
:10227600CB7F007EC07DA87C001226AAEFF40490D6
:102286007042F090709EE0FFC43354E0FF9070A956
:10229600E024182F907043F07B017A7079407D041A
:0F22A600122C187B017A7079407D04122C1822BB
:062D46007F48122B5B2206
:101D7C009070E9EBF0A3EAF0A3E9F0907000EDFFAE
:101D8C007E017480F0A3E4F0C5827002158314C543
:101D9C0082C9C582C9CAC583CAE0F8A3C9C582C9AC
:101DAC00CAC583CAEEFBE8C313DBFCF5F0E045F0D3
:101DBC00F0A3E045F0F0A37407C39EFB6007E8C3F3
:101DCC0033DBFC8001E8D2E7F0A3C2E7F0C58270F8
:101DDC0002158314C582BE0715A3A37480F0A3E477
:101DEC00F0C5827002158314C5827E0180010EDD60
:101DFC00A0EF75F008A4240675F00784C333FF2206
:0C1E0C009070E9E4F0A3F0A3F0FDFF22C9
:102C1800121D7CCEEFCE7F487C707D00CBEECBC200
:052C2800011227B0229B
:101FDA00C0D075D00890709CE07002A3E070030234
:101FEA00206B740A2572F57290709BE065727071AD
:101FFA00F5729070407415F0A37401F0E573A3F0C4
:10200A00E574A3F0E56160080574E5747002057370
:10201A00E529907044F0E52AA3F0E52BA3F0E52C1E
:10202A00A3F0E52DA3F0E52EA3F0E52FA3F0E5300C
:10203A00A3F0E531A3F0E532A3F0E533A3F0E534EC
:10204A00A3F0E535A3F0E536A3F0E537A3F0E538CC
:10205A00A3F0A3E540F07B017A7079407D15122C3C
:04206A0018D0D02298
:102AC4000000CC01D8011400F0013C002800E4010E
:102AD400A0016C007800B40150009C0188014400FE
:050026007EFF7FFF22B8
:1020EB00CBEFCBCAEECAC9EDC9E9540FFFEAEB6FD0
:1020FB00540F25E0FFE433FE74C42FF582EE342A2F
:10210B00F583EAC4F854F0C868FEEBC4540F48FFDB
:10211B00EE540FFEE4936EFA7401936FFBCFE9CF8D
:10212B00EFC4540F540FFFEAEF6B540F25E0FFE49D
:10213B0033FE74C42FF582EE342AF583EAC4F854C7
:10214B00F0C868FEEBC4540F48FFEE540FFEE49347
:0C215B006EFA7401936FFBCEEACEFF22F7
:072D2D00EEF4FEEFF4FF22BB
:10251F00FF2D68FF2CFAFF2D04FF2AA3FF2D4CFF80
:10252F002A5EFF2D52FF2D6CFF2C9AFF2D58FF2A8C
:10253F00E4FF2BC0FF2D70FF2D77FF2D78FF2D7936
:10254F00FF2D7AFF2D7BFF2D7CFF2D7DFF2D7EFF35
:10255F002D7FFF2D80FF2D81FF2D82FF2D83FF2DDE
:10256F005EFF2D5EFF2D5EFF2D5EFF2D5EFF2D5E4C
:0F2C8B00D296D29775D8C575DBECD2BDD2AD22EB
:102B5B00E4F5688F66D21BD2DDFF122996EF64185D
:0B2B6B006004EFB44003D38001C322DC
:1027B0009070E9ECF0A3EDF08C838D82787AEBFEDB
:1027C0006006E0F6A308DEFA8B688F66D21BD2DDC6
:1027D00030010DCFEBCF1229969070EBEFF0800512
:0B27E000E49070EBF09070EBE0FF2243
:102731009070EFEBF0A3EAF0A3E9F0CEEFCEA3E0C7
:10274100FFF5688E66D21BD2DD122996E4FE9070E9
:10275100F2E06E601D747A2EF8E6FD9070EFE0FBFA
:10276100A3E0FAA3E0F98E82758300ED1203D30E84
:0327710080DC22E7
:10299600CEEFCEE4F563EE2402FDE433FCE5636D91
:1029A6007001EC6010756428D564FD201B03AF67C9
:0B29B60022056380E175D8D57F002268
:042D680075D8D52223
:0A2CFA008566DA75D8C5E4F5652299
:0A2D04008566DA75D8C5E4F565228E
:102AA300C0D075D010E568700775D8D5C21B800EED
:102AB300AF650565747A2FF8E6F5DA75D8C5D0D019
:012AC30022F0
:062D4C0075D8D5C21B2260
:102A5E00C0D075D010E5656568700775D8D5C21BF6
:102A6E00800EAF650565747A2FF8E6F5DA75D8C570
:032A7E00D0D02293
:062D520075D8D5C21B225A
:042D6C0075D8E5220F
:0F2C9A00E568700775D8D5C21B800375D8C522B1
:062D580075D8D5C21B2254
:102AE400C0D075D010AF650565747A2FF8A6DAE505
:102AF400656568700575D8C1800375D8C5D0D022C6
:102BC000C0D075D010AF650565747A2FF8A6DA7598
:072BD000D8D5C21BD0D022B2
:042D700075D8D5221B
:012D77002239
:012D78002238
:012D79002237
:012D7A002236
:012D7B002235
:012D7C002234
:012D7D002233
:012D7E002232
:012D7F002231
:012D80002230
:012D8100222F
:012D8200222E
:012D8300222D
:062D5E0075D8D5C21B224E
:03002B0002277435
:10277400C0E0C0F0C083C082C0D075D01085D967D6
:10278400E5D9131313541F75F003A4241FF582E431
:102794003425F583E493740193FA740293F91206D1
:0C27A40060D0D0D082D083D0F0D0E032E2
:03000000022CDAF5
:0C2CDA00787FE4F6D8FD7581D102206EF1
:1003BA00BB010689828A83E0225002E722BBFE0241
:0903CA00E32289828A83E4932274
:1003D300F8BB010DE58229F582E5833AF583E8F060
:1003E300225006E92582C8F622BBFE05E92582C80C
:0203F300F222F4
:1003F500EFF88DF0A4FFEDC5F0CEA42EFEEC88F04D
:04040500A42EFE2201
:10040900BC000BBE0029EF8DF084FFADF022E4CCD7
:10041900F875F008EF2FFFEE33FEEC33FCEE9DECA0
:10042900984005FCEE9DFE0FD5F0E9E4CEFD22EDE6
:10043900F8F5F0EE8420D21CFEADF075F008EF2F30
:10044900FFED33FD4007985006D5F0F222C398FD21
:050459000FD5F0EA22BE
:10045E00C2D5EC30E709B2D5E4C39DFDE49CFCEEB9
:10046E0030E715B2D5E4C39FFFE49EFE120409C324
:10047E00E49DFDE49CFC800312040930D507C3E41F
:06048E009FFFE49EFE2228
:10049400C5F0F8A3E028F0C5F0F8E58215827002F3
:0604A4001583E038F02290
:1004AA00A3F8E0C5F025F0F0E58215827002158305
:0604BA00E0C838F0E82262
:1004C000E88FF0A4CC8BF0A42CFCE98EF0A42CFCDB
:1004D0008AF0EDA42CFCEA8EF0A4CDA8F08BF0A459
:1004E0002DCC3825F0FDE98FF0A42CCD35F0FCEBB8
:1004F0008EF0A4FEA9F0EB8FF0A4CFC5F02ECD397D
:0F050000FEE43CFCEAA42DCE35F0FDE43CFC22E9
:10050F0075F008758200EF2FFFEE33FECD33CDCCA3
:10051F0033CCC58233C5829BED9AEC99E582984026
:10052F000CF582EE9BFEED9AFDEC99FC0FD5F0D603
:10053F00E4CEFBE4CDFAE4CCF9A88222B800C1B92D
:10054F000059BA002DEC8BF084CFCECDFCE5F0CB6B
:10055F00F97818EF2FFFEE33FEED33FDEC33FCEBA4
:10056F0033FB10D703994004EB99FB0FD8E5E4F95F
:10057F00FA227818EF2FFFEE33FEED33FDEC33FC4C
:10058F00C933C910D7059BE99A4007EC9BFCE99A40
:10059F00F90FD8E0E4C9FAE4CCFB2275F010EF2F85
:1005AF00FFEE33FEED33FDCC33CCC833C810D70785
:1005BF009BEC9AE899400AED9BFDEC9AFCE899F8C0
:0E05CF000FD5F0DAE4CDFBE4CCFAE4C8F92253
:1026AA00C2D5E830E70FB2D5E4C39BFBE49AFAE45B
:1026BA0099F9E498F8EC30E717B2D51226E012053A
:1026CA004BE4C39BFBE49AFAE499F9E498F8800393
:1026DA0012054B30D50DE4C39FFFE49EFEE49DFD39
:0426EA00E49CFC224E
:1005DD00EB9FF5F0EA9E42F0E99D42F0EC6480C895
:0605ED0064809845F02235
:1005F300EB9FF5F0EA9E42F0E99D42F0E89C45F05E
:0106030022D4
:10060400E8600FECC313FCED13FDEE13FEEF13FFD4
:03061400D8F122F8
:0C061700ECF0A3EDF0A3EEF0A3EFF02256
:10062300A8828583F0D083D08212063A12063A124A
:10063300063A12063AE473E493A3C583C5F0C5836F
:10064300C8C582C8F0A3C583C5F0C583C8C582C821
:010653002284
:0C065400A42582F582E5F03583F58322B1
:060660008A838982E47325
:10005E00E56924C1F582E43470F583E005692290E8
:10006E0070BE3009039070C1E475F0011206B30240
:10007E0003BA2002E97F2ED2028018EF540F24908B
:10008E00D43440D4FF30060BEF24BFB41A00500313
:10009E002461FFE56A6002156A056DE56D70020563
:1000AE006C30090E9070BEE475F0011206B3EF02CB
:1000BE000693022D0E7403D2098003E4C209F5697A
:1000CE009070BE1206CAE4F56AF56CF56DE56A60CD
:1000DE00077F201200A180F5F56BC203C202C20495
:1000EE00C205C207C208C20A12006DFF700D3009A8
:1000FE00057F001200B2AF6DAE6C22B42561C2D581
:10010E00C20612006DFF24D0B40A00501C75F00A0E
:10011E0020D50DC56AA4256AF56A7002D20580E065
:10012E00C56BA4256BF56B80D724CFB41A00EF50A6
:10013E0004C2E5D2060202ACD20380C4D20280BE53
:10014E00D20480BAD2D580B8D20780B27F201200F6
:10015E00A12004077401B56A0040F112005EFF127F
:10016E0000A10200DBD20AD208809312005EFB12BD
:10017E00005EFA12005EF94A4B700679787A037BBC
:10018E00FF200433E56A602FAF6BBF00011F7E00B6
:10019E008E8275830012066660050EEE6F70F1C2D8
:1001AE00D5EBC0E0EAC0E0E9C0E0EE1202F0D0E02C
:1001BE00F9D0E0FAD0E0FB1203BAFF60A5EBC0E085
:1001CE00EAC0E0E9C0E01200A1D0E02401F9D0E0DD
:1001DE003400FAD0E0FBE56B60DDD56BDA80837B13
:1001EE00FF7A0279ECD2048098791080027908C2E5
:1001FE0008C20A8008D2D5790A8004790AC2D5E4E9
:10020E00FAFDFEFF12005EFC7B0820031312005E57
:10021E00FD7B1030020A12005EFE12005EFF7B2094
:10022E00EC3382D592D55013C3E43002069FFFE41F
:10023E009EFEE42003039DFDE49CFCE4CBF8C20388
:10024E00EC700CCFCECDCCE824F8F870F38017C349
:10025E00EF33FFEE33FEED33FDEC33FCEB33FB9966
:10026E004002FB0FD8E9EB300305F8D0E0C448B2EA
:10027E0003C0E00AEC4D4E4F78207B0070C2EAC0FE
:10028E00E01202F2D0F0D0E0200304C4C0E0C4B209
:10029E0003C0F012008AD0F0D5F0EB0200DB12069C
:1002AE00D301795301F758014A4C01464201FB4FE5
:1002BE00020344020349015F4302095501ED460161
:1002CE00ED4501ED47039B50014E2D01522E017558
:1002DE002B01562301732003862A0000016D3F3F38
:1002EE003F00790AA2D5200514300709B91002047F
:1002FE0004B9080104A2D5200802500104200466A6
:02030E00920457
:10031000B56A005032C0E07F203005177F30A2045C
:1003200072087207500D120347C204C208C2077F49
:1003300030800F300703E9C0E01200A1300703D07E
:10034000E0F9D0E0B56ACE3007177F30B9100C1253
:1003500000A17F583006077F788003B90803120098
:10036000A13004057F2D0200A17F20200AF87F2BF9
:100370002008F322920480CF286E756C6C29002D22
:1003800050434958D20312005E3003F8C203786A22
:1003900030D504D202786BF602010C12005E240301
:1003A000B405004001E490037F93120092743A1266
:0A03B0000092D205756A040201F7FD
:102C2D00EFC394094006EFC3940E4004EFB42003A4
:052C3D00D38001C32259
:1023F3009070E9EBF0A3EAF0A3E9F09070ECE0FB56
:10240300A3E0FAA3E0F91203BAFE9070E9E0FBA39C
:10241300E0FAA3E0F91203BAFD6E702AED600E90A4
:1024230070EF74FFF5F012049445F070037F0022FF
:102433009070EAE475F0011204949070EDE475F085
:102443000112049480B5D3EE6480F8ED6480984063
:07245300037F01227FFF223D
:102B3F00E94A4B7001221203BAFF6D700122EF7048
:0C2B4F0004FBFAF92209E970ED0A80EAA3
:101599009070FAEBF0A3EAF0A3E9F09070FAE0FB9F
:1015A900A3E0FAA3E0F91203BAFF122C2D500C9014
:1015B90070FBE475F00112049480E0D2019070FA96
:1015C900E0FBA3E0FAA3E0F91203BAFF642B60047D
:1015D900EFB42D1D9070FAE0FBA3E475F00112043D
:1015E900AAA9F0FA1203BA642D6003D38001C39249
:1015F900019070FD120623000000009070FAE0FBD4
:10160900A3E0FAA3E0F91203BAFF122C7A506A7F19
:101619000A7E007D007C009070FDE0F8A3E0F9A34C
:10162900E0FAA3E0FB1204C0C8ECC8EDC0E0EEC0CC
:10163900E0EFC0E09070FAE0FBA3E0FAA3E0F91252
:1016490003BAFF3395E0FEEF24D0FFEE34FFFEE44A
:10165900FCFDD0E0FBD0E0FAD0E0F9EB2FFFEA3E49
:10166900FEED39FDEC38FC9070FD1206179070FB09
:10167900E475F00112049480823001109070FDE04D
:10168900FCA3E0FDA3E0FEA3E0FF80119070FDE064
:0E169900FCA3E0FDA3E0FEA3E0FF1206A522E5
:1019AB00907107EBF0A3EAF0A3E9F0907107E0FB6D
:1019BB00A3E0FAA3E0F91203BAFF122C2D500C90FE
:1019CB007108E475F00112049480E0D20190710764
:1019DB00E0FBA3E0FAA3E0F91203BAFF642B600467
:1019EB00EFB42D1D907107E0FBA3E475F001120419
:1019FB00AAA9F0FA1203BA642D6003D38001C39233
:101A0B0001E490710AF0A3F0907107E0FBA3E0FAF8
:101A1B00A3E0F91203BAFF122C7A503F907107E042
:101A2B00FBA3E0FAA3E0F91203BAFF3395E0FEEF54
:101A3B0024D0FBEE34FFFA90710AE0FEA3E0FF7CAA
:101A4B00007D0A1203F5EF2BF0EE3A90710AF0903D
:101A5B007108E475F00112049480AD30010A9071A5
:101A6B000AE0FEA3E0FF800F90710AE0FEA3E0FF07
:081A7B00C3E49FFFE49EFE227C
:10066600BB010CE58229F582E5833AF583E0225049
:1006760006E92582F8E622BBFE06E92582F8E22293
:0D068600E58229F582E5833AF583E49322AD
:10069300BB010689828A83F0225002F722BBFE0146
:0206A300F32240
:0E06A500C3E49FFFE49EFEE49DFDE49CFC2266
:1006B300F8E0FBA3A3E0F925F0F0E58215827002D0
:0706C3001583E0FA38F02274
:0906CA00EBF0A3EAF0A3E9F02231
:1006D300D083D082F8E4937012740193700DA3A3B6
:1006E30093F8740193F5828883E4737402936860CA
:0606F300EFA3A3A380DFCA
:102C7A00EFC394304009EFC3943A5003D38001C3A1
:012C8A002227
:00000001FF
